:020000040000FA
:0200000088284E
:020008007A2854
:02000E008A0165
:100010001708820712281F282C2839284628532819
:1000200060286D28180882074134543444343E3423
:100030002234313422343B340D340A34003418086D
:1000400082074134543444343E342234323422342E
:100050003B340D340A3400341808820741345434D8
:1000600044343E342234333422343B340D340A34A5
:100070000034180882074134543444343E34223466
:10008000343422343B340D340A34003418088207E7
:100090004134543444343E342234353422343B34F5
:1000A0000D340A340034180882074134543444347F
:1000B0003E342234363422343B340D340A34003496
:1000C000180882074134543444343E3422343734DF
:1000D00022343B340D340A3400341808820741348A
:1000E000543444343E342234383422343B340D34D6
:1000F0000A3400340B119B0F872805109C19051436
:100100009C0A1E301C02031C87289C011D14090038
:10011000031E8E28831D8E280000000083018B01A2
:1001200083168F30810010308500FF3086008312E7
:1001300085010516970198019A019B019C019D017B
:10014000A0308B0064001D1CA2288B131D10061804
:10015000D0289A0A1F301A02031CC2289A0185145B
:100160004130E1205430E1204830E1200D30E120E1
:100170000A30E1208510970A08301702031CDE2898
:100180009701DE2805159801143099000720003EDC
:100190000319CE28E120980A990BC6280511DE28FC
:1001A00085144130E1205430E1204830E1200D3009
:1001B000E1200A30E120851097019A01A0308B00E0
:1001C000A2289100083092008511FA200310910CAA
:1001D00003188515031C8511F420920BE62885155C
:1001E000FA2000341F30FD281D30FD282F30FD2857
:1001F0001030FD282230FD2821309300930BFE287B
:10020000003420342034623479343A3420343234A7
:1002100030343034383420345334743461346E34F0
:100220006B346F34763469346334203447346F343C
:10023000723461346E3420346434693470346C3414
:100240002E3469346E3467342E3465346C342E3475
:100250002034203445342D346D34613469346C34A9
:100260003A34203467346F34723461346E3473340A
:10027000743461344034453455346E3465347434E8
:100280002E34793475342034203420342034203412
:1002900020342034203420342034203420342034BE
:02400E000500AB
:00000001FF
